:10000000A4C00000B2C00000B0C00000AEC000003C
:10001000ACC00000AAC00000A8C00000A6C000003C
:10002000A4C00000A2C00000A0C000009EC000004C
:100030009CC000009AC0000098C0000029C30000C6
:100040006AC2000092C0000090C000008EC0000094
:100050008CC000008AC0000088C0000086C000007C
:1000600084C0000082C0000080C000007EC000008C
:100070007CC00000A301A501A701A901AB01BA0141
:100080003002BC01C601CC01DA01DF010001000031
:10009000BA001200020000CC001200030000DE00D3
:1000A0000401030904E20028020309040C011E03F1
:1000B0000309042C011C00000000120100020000D2
:1000C0000040CDAB09FA0001010203010902120050
:1000D000010100C0320904000000FF010100040317
:1000E000090428035B004D0061006E007500660086
:1000F00061006300740075007200650072002000EA
:1001000068006500720065005D0000001E035B0072
:10011000500072006F0064007500630074002000DE
:1001200068006500720065005D0000001C035B0054
:10013000530065007200690061006C0020006800D7
:100140006500720065005D00000011241FBECFEF46
:10015000D4E0DEBFCDBF12E0A0E0B1E001C01D924F
:10016000A632B107E1F790D37EC584C3582F5198CA
:1001700098E080E0232D31E0422F00004150E9F764
:100180003150D1F7509832E0422F00004150E9F74A
:100190003150D1F7880F49998160509A31E0422F50
:1001A00000004150E9F73150D1F7915021F751113A
:1001B00001C0519A332D91E0232F00002150E9F71F
:1001C0009150D1F75098332D93E0232F0000215008
:1001D000E9F79150D1F7509A332D91E0232F000089
:1001E0002150E9F79150D1F7712C612C5198089565
:1001F00098E0232D31E0422F00004150E9F73150C3
:10020000D1F787FF02C0519801C0519A880F31E0A1
:10021000422F00004150E9F73150D1F7509832E0B9
:10022000422F00004150E9F73150D1F7509A9150D8
:1002300009F75198232D82E0922F00009150E9F7A1
:100240008150D1F75098232D82E0922F00009150D9
:10025000E9F78150D1F799B19270509A332D81E02E
:10026000232F00002150E9F78150D1F7712C612C28
:1002700081E0911101C080E008955098232D81E024
:10028000922F00009150E9F78150D1F7612C712C29
:1002900051980895519A232D81E0922F000091509A
:1002A000E9F78150D1F7612C712C509A0895809113
:1002B000E80080FFFCCF08950895A0E0B0E0E2E6FA
:1002C000F1E09EC41092020123E031E001C09E01E2
:1002D000E9018991982F907F903161F118F4992369
:1002E00039F0F5CF903509F4BDC0903F81F70FC1CB
:1002F0008F70883071F018F4813049F705C089306B
:1003000051F08F3021F709C085E08A95F1F70000A0
:10031000DECF5F98DCCF5F9ADACF80910201A82F01
:10032000B0E0F9019181AD5FBE4F9C938F5F8093E8
:10033000020142C08F7090E08C30910540F6865CDF
:100340009F4FFC018AC43A98C2CF3A9AC0CF4298D4
:10035000BECF429ABCCF80910201E82FF0E096B167
:1003600092FB992790F9ED5FFE4F90838F5F80930A
:100370000201ADCF8FDFABCFF09002010F2D10E067
:10038000E9012296F901818133DF0CC0F09002016E
:100390000F2D10E080E005C0F09002010F2D10E05D
:1003A00081E0E4DEF801ED5FFE4F8083F394F0928C
:1003B00002018DCFF9013180E901229688CFF90140
:1003C000E180EE0CD280F380E901249663DFC090D7
:1003D00002010C2D10E08E2D0BDFF801ED5FFE4FBA
:1003E0008083C394C09202018E01CC2ECD0C04C038
:1003F000F80181918F01FCDEC012FACFCD0DD11D25
:100400003CDFFF2009F463CF45DFD09002010D2DC2
:1004100010E08E2D8160ECDEF801ED5FFE4F8083F1
:10042000D394D09202010DC0E09002010E2D10E095
:1004300080E09CDEF801ED5FFE4F8083E394E09264
:100440000201FA9489F7F09002010F2D10E081E08B
:100450008DDEF801ED5FFE4F8083F394F092020190
:100460000CDF35CFF901418132961CC0809101012A
:100470002091000190E001968F77992730E0821754
:100480009307A1F38191A0910101B0E0AB57BE4F5A
:100490008C938091010190E001968F77992780934A
:1004A000010141504111E2CF80910201E82FF0E0BB
:1004B00090910502ED5FFE4F90838F5F8093020164
:1004C00080910201E82FF0E0ED5FFE4F10828F5F18
:1004D00080930201E6E0F2E09081218132968091E2
:1004E0000201A82FB0E0AD5FBE4F2C938F5F8093C9
:1004F000020180910201A82FB0E0AD5FBE4F9C9336
:100500008F5F8093020182E0EE31F80729F7CDB7C3
:10051000DEB7E8E091C31F920F920FB60F9211243D
:100520002F938F939F93EF93FF934D9B0CC010924B
:100530001F0280910802909109020196909309028E
:100540008093080207C080911F028A3018F48F5FE1
:1005500080931F024E9B0CC01092210280910C02CE
:1005600090910D02019690930D0280930C0207C0AA
:10057000809121028A3018F48F5F809321021C9BA6
:100580000CC01092230280911002909111020196EA
:10059000909311028093100207C0809123028A3049
:1005A00018F48F5F8093230290911F0280910502BF
:1005B0009A3010F4826001C08D7F80930502909183
:1005C0002102809105029A3010F4886001C0877F73
:1005D0008093050290912302809105029A3010F4D5
:1005E000806201C08F7D809305023F9A549A47989C
:1005F0005C9A109224025A982E9846989091010184
:100600008091000198130CC0109225028091120273
:1006100090911302019690931302809312022EC0C0
:10062000E0910001F0E0EB57FE4F20818091000146
:1006300090E001968F7799278093000120932502FF
:1006400020FF02C02D9A01C02D98259A922F9870F4
:10065000822F807221FD02C0459A01C045989111F8
:1006600002C02F9A01C02F98882311F05B9A01C015
:100670005B9827FF02C0449A01C04498FF91EF9114
:100680009F918F912F910F900FBE0F901F901895F3
:100690001F920F920FB60F9211242F933F934F93F7
:1006A0005F936F938F939F934D9B0CC010921E028C
:1006B0008091060290910702019690930702809321
:1006C000060207C080911E028A3018F48F5F809363
:1006D0001E024E9B0CC01092200280910A02909143
:1006E0000B02019690930B0280930A0207C080913F
:1006F00020028A3018F48F5F809320021C9B0CC06C
:100700001092220280910E0290910F020196909316
:100710000F0280930E0207C0809122028A3018F4E3
:100720008F5F8093220290911E02809105029A3081
:1007300010F4816001C08E7F8093050290912002A9
:10074000809105029A3010F4846001C08B7F809301
:10075000050290912202809105029A3010F4806186
:1007600001C08F7E809305023F9A549A479A5C9805
:10077000809124028F5F809324024091250243FBE5
:10078000662760F945FB552750F980911A02909130
:100790001B02019690931B0280931A02809105021E
:1007A00041FB992790F941FF03C081FD17C002C0AA
:1007B00080FD14C042FF4DC02091140230911502FB
:1007C000992319F081E090E002C08FEF9FEF820F34
:1007D000931F9093150280931402469A809105020C
:1007E000662319F083FD17C002C082FD14C044FFC8
:1007F00032C02091160230911702662319F081E071
:1008000090E002C08FEF9FEF820F931F909317022B
:10081000809316022E9A80910502552319F085FFC8
:1008200003C01CC084FD1AC046FF17C020911802E7
:1008300030911902552319F081E090E002C08FEF4A
:100840009FEF820F931F90931902809318025A9A78
:1008500005C04698C3CF2E98DECF5A989F918F91AE
:100860006F915F914F913F912F910F900FBE0F901D
:100870001F9018951F920F920FB60F9211240F9090
:100880000FBE0F901F901895F89480E88093610038
:10089000109261008FEF8093840180EA8093D800EA
:1008A0001092630086E089BD09B400FEFDCF80E8A8
:1008B0008093D8001092E00088E08093E20081E00D
:1008C00080938401579A5F9A8BB18C7F8BB98AB1E0
:1008D0008C7F8AB98AE0382E82E0809380008AE19A
:1008E000809381008AEF90E0909389008093880044
:1008F00081E090E090938B0080938A0084EF91E0F8
:10090000909387008093860086E080936F0010921A
:10091000E2003F9A4798549A5C988AB18F798AB9D5
:1009200024982D98259A459A3D9A469A3E9A2F9A50
:10093000279A2E9A269A5B9A539A5A9A529A449ACE
:100940003C9A789492EF292E2EEFA22E3BEFB32EF5
:10095000992493944EE1442E52E0552E61E2862E66
:100960001092E9008091E8008F7529F48091EE00E3
:10097000807609F421C11092E9008091E80083FF9C
:1009800016C19091F1008091F1002091F100309119
:10099000F100D32F30E0C32F6E01C22A2091F10065
:1009A0003091F1004091F1005091F100152F00E0DD
:1009B000B801642BAB012092E800863009F052C0E8
:1009C00003C08092EB00F3C0F32EE12CC701822B11
:1009D0009C01A6E08CE890E0FC01659174916C1597
:1009E0007D0509F007C0FC0132966591749162178C
:1009F000730711F0079612C0FC013496659174914B
:100A00009B01FC01369684914F3F510519F010F07F
:100A10004FEF50E0481728F4842F03C0A150E1F6AF
:100A2000D0CF9091E800492F4570D9F392FDBFC017
:100A3000982F813408F090E4A901692F07C0FA01CA
:100A40004F5F5F4FE491E093F10061506111F7CF88
:100A5000290F311D891BA092E8008111E2CF90344B
:100A600001F3A5C0853041F4A092E80020DC689431
:100A7000C7F8C092E3009BC0893051F5911197C02F
:100A8000C0928301A092E80086EB90E041E04093A1
:100A9000E9009C012F5F3F4FFC0154915093EB0004
:100AA000552359F0F90124912093EC00FC01329672
:100AB0000396E491E093ED0001C0C9014F5F45301A
:100AC00031F74092EA001092EA00509284016FC020
:100AD000883049F4903809F06AC0E9DB80918301DD
:100AE0008093F10062C0811106C0E1DB1092F10039
:100AF0001092F1005AC0833CB1F48091E800982F25
:100B00009570D9F382FD53C080E008C0E82FF0E073
:100B1000ED5FFE4F90819093F1008F5F9091020105
:100B20008917A0F342C0843CA9F48091E80082FFB9
:100B3000FCCF80E090E007C02091F100FC01ED5F68
:100B4000FE4F2083019684179507B1F7B6DBB0926C
:100B5000E8002BC0853C09F580E09091E80092FF09
:100B6000FCCF942F413408F090E4292F280F08C0BF
:100B7000E82FF0E03091F100ED5FFE4F30838F5FA2
:100B80008213F6CF491BB092E800A092E800411111
:100B9000E4CF903411F391DB0AC0893C41F4809199
:100BA000E800982F9570D9F382FFA092E800809119
:100BB000EE008F798093EE008091E10083FFD0CE2C
:100BC0008091E1001092E10083FFCACE1092E9000B
:100BD0009092EB001092EC0082E38093ED00109273
:100BE000F0001092830190928401BACE2F923F922E
:100BF0004F925F926F927F928F929F92AF92BF922D
:100C0000CF92DF92EF92FF920F931F93CF93DF93D8
:100C1000CDB7DEB7CA1BDB0B0FB6F894DEBF0FBE35
:100C2000CDBF09942A88398848885F846E847D8482
:100C30008C849B84AA84B984C884DF80EE80FD8084
:100C40000C811B81AA81B981CE0FD11D0FB6F894FA
:100C5000DEBF0FBECDBFED010895EE0FFF1F059063
:0A0C6000F491E02D0994F894FFCF01
:00000001FF
